:030000000219FDE5
:03000B000200AA46
:03002B0002015C73
:03005B000202F6A8
:030073000202E3A3
:1000800002030406080C10182030406080040608A3
:100090000C10182030406080A0C00003070F1F0D17
:1000A0000D04050D050305030302C2AFC0D0C0E077
:1000B000206214E5256009E473E525F4F58AD2622F
:1000C000D0E0D0D0D2AF3285268AC262E526F46075
:1000D0002F30682520720DD0E0D0D0D295D293D2A7
:1000E00097D2AF32D295D293D297206F0C20650968
:1000F000740CD5E0FDE57B4290D0E0D0D0D2AF3299
:10010000758A00C28DD26201F901B9306805206597
:1001100002C29501B9306805206502C29701B93065
:100120006805206502C29301B9C29430680A20654F
:10013000077401D5E0FDC29501B9C29630680A2066
:1001400065077401D5E0FDC29701B9C29230680A13
:100150002065077401D5E0FDC29301B9C2AFC2ADFD
:1001600053E6EFC0D0C0E0D2D3D2AFC2CEE52A6012
:100170000720744F152A21C37800790020742EE5DA
:1001800080307E01F430E50278FF53DACF207E0321
:1001900043DA20307E0343DA10C2D8C271E58030E2
:1001A0007E01F430E50279FFC3E89970CB3061033A
:1001B000752A18207403752A18885CD270E86003C9
:1001C000755F0020740DE52B6004152B21D343DAF5
:1001D00001C2D82070024142A85C206102C2702096
:1001E00074367982B70431C3E894F0400374F0F8B0
:1001F000E8C4540F28F87984B703024118C313C325
:10020000138721200802C313200A06C3C898F841A7
:100210001828F8500374FFF88822E52D5406602250
:10022000206B1FE536C333C333F8E564C313C31330
:10023000F9C3952240028922E82522F52250037550
:1002400022FF7882B60459852224A824C3E5249588
:10025000614002A861C3E895634002A8638825E570
:100260006670024193C3E8AA669A5003E8FAE4F97B
:10027000EAC333FBE568F45B29400D2567F8E567C1
:1002800060021567400B41930AC3E5679A50020567
:100290006778FF8826C26FC3E52694F84002D26FC4
:1002A00020CF0AD0E0D0D043E610D2AD32C2CF0585
:1002B0003A7801E52A6005307402152AC3E55C949A
:1002C000014005755F0041D9756000756900E55F03
:1002D0002401F55F5003755FFFD0E0D0D043E610F6
:1002E000D2AD32C2AF53E67F7592FA7593FFC2600A
:1002F000759104D2AF32C2AF53E6EFC2ADC0D0C0E9
:10030000E0C0F0D2D3D2AFA8FBA9FCC2D8307102B2
:10031000615D53DACF207E0343DA10307E0343DA87
:1003200020D271E580307E01F420E5026134882717
:100330008928A18A53DACF207E0343DA20307E0356
:1003400043DA10C2D8C271307402A1767800E58019
:10035000307E01F430E502A176885CA15E53DACFED
:10036000207E0343DA20307E0343DA10C27120611D
:1003700002813653DACF207E0343DA10307E034306
:10038000DA20C2D8D27188578958C3E89555F8E960
:100390009556F97B007E087A00C3E8948CE99400B6
:1003A0005005755B008128882178A2E6A821605558
:1003B000C3E894C8E994005008E4D2E4FB7A0A81C7
:1003C00003C3E89468E994015008E4D2E3FB7A0F90
:1003D0008103C3E894D0E994025008E4D2E2FB7AA6
:1003E0001E8103C3E894A0E994055008E4D2E1FB20
:1003F0007A3C8103C3E89498E994085008E4D2E079
:10040000FB7A787E00C3E89559FCE9955AFD30E700
:100410000AECF42401FCEDF43400FD755B00C3EC40
:100420009AED9E5003755B018859895A8557558509
:1004300058567802A15EC3E89527F8E99528F93067
:100440007C02A142307B02A142307A02A13B20759E
:10045000028159E9FDE8FC8178E9C313F9E813F852
:10046000307902A13BE9C313F9E813F8307802A10F
:0F0470003BE9C313FDE813FC20612CC3EC941C83
:10047F00ED94024002818FED701EC3EC94C85018AA
:10048F000529E52970021529C3E529940A5002A10F
:10049F0076755C00D270A176E529600215297888FF
:1004AF00E6F97400207F087896B90302789EE62457
:1004BF00FAFEE43400FFC3EC9EFCED9FFD9208B9F9
:1004CF000310A2085007207609D27681E130760218
:1004DF00C276A2085016B9030DECF42401FCEDF41A
:1004EF003400FD0204FB78007900A142B90315EC3A
:1004FF0033FCED33FDC3EC940AFCED9400FD500486
:10050F007C007D00C3EC94FFED9400400678FF79EA
:10051F0000A142EC8572F0A4C5F0A2F733F8790080
:10052F00400302055E78FF790002055EE9C313F907
:10053F00E813F8307C0EE9600278FFC3E81338F84F
:10054F00E43400F9C3E894FFE99400400278FF888F
:10055F005CD270206102A176741FF4552F4BF52FDA
:10056F00C274EB7002D274752A18307403752A0A9C
:10057F00306102A18A20740353DAFE207403752BB5
:10058F0006D0F0D0E0D0D0D2AD43E61032790102E0
:10059F0005BA79030205BA790A0205BA791E02056E
:1005AF00BA79640205BA79C80205BA7817E4D5E0BA
:1005BF00FDD8FAD9F6227A147B780205E17A107BFE
:1005CF008C0205E17A0D7BB40205E17A0B7BC80240
:1005DF0005E1E573D5E001227902E4C296D5E0FD8D
:1005EF00C297D5E0FDD297D5E0FDD296D5E0FDE9D3
:1005FF0020E002C29530E002C293E573D5E0FDE939
:10060F0020E002D29530E002D2937496D5E0FDD966
:10061F00C9EAF8D5E0FDD8FBDBB8C29622C37C004F
:10062F007D0075F00005F0EA33FAEB33FB50F6EB83
:10063F0013FBEA13FAC3E9FFE8FEE89AF8E99BF91E
:10064F005004EFF9EEF8B3EC33FCED33FDD5F0DFEA
:10065F00EDF9ECF822E889F08A20D2D4F8A9F07BE2
:10066F000030F70B7BFFF42401F8E9F43400F9E8CC
:10067F008520F0A4ADF0F8E98520F0A4AFF0FEEDF1
:10068F002EF974003FFA7C04C3EA13FAE913F9E870
:10069F0013F8DCF48BF030F70AE8F42401F8E9F4EE
:1006AF003400F9E889F0C2D4F8A9F0227882B604B0
:1006BF0003020716C3E55C940140030206E085229E
:1006CF0024E4F544F545F546F547F548C26E0207B3
:1006DF00167882E6FCD26EE522F523783879C7AA20
:1006EF0040AB41C3EB13FBEA13FAEC146013C3EBFB
:1006FF0013FBEA13FAEC14146007C3EB13FBEA13B2
:10070F00FAD12C8844894522C3E5449523F8E54561
:10071F009400F9500CC3E89480E994FF4016020747
:10072F0047C3E8947FE994005003020747787F7925
:10073F0000020747788079FF8849894A22E54925D1
:10074F0046F8E54A3547F9854A20E4300701F43584
:10075F0048FA30E709C3EA94F04015020785C3EA67
:10076F00940F500302078578FF79FF7A0F020785F0
:10077F00780079007AF0C3E5249561500AC37401BB
:10078F009524500B0207A3E54A20E70E0207A3E5C5
:10079F004A30E706884689478A482278A5E6FAC391
:1007AF00E54933F8E54A33F9D164E930E70BC3E89B
:1007BF009480E994FF4013E1DDC3E8947FE994004E
:1007CF005002E1DD787F7900E1DD788079FFE82064
:1007DF00E715C3E52398F84009C3E89401400302E5
:1007EF0008047801020804E8F424012523F84003E3
:1007FF0002080478FF884B2278A6E6FAA847A94892
:10080F00120664E930E70CC3E89401E994FF40163F
:10081F00020839C3E894FFE99400500302083978BD
:10082F00FF7900020839780179FFE920E715C3E560
:10083F004B98F84009C3E89401400302086078011F
:10084F00020860E8F42401254BF8400302086078A1
:10085F00FF88242278FF20692879A1E76023E541EA
:0E086F00601F74FF8541F0848539F0306A0304
:10087D0075F005A4F8C5F0600278FFC3E8956450E3
:10088D0002A864886322C3E5409440E5419401E5E4
:10089D006350031401A4046002F563220208AC2224
:1008AD0075E890227883E6FF30EDF9A8BDA9BE0565
:1008BD0070C3E57094084052757000E9FA79A0E7AD
:1008CD006044EA7007E571601B0208E5C3E89571A5
:1008DD006010E5715006600C140208F10460F90215
:1008ED0008F1E571F571C3946D401B7561C0C3943A
:1008FD00044013756180C39404400B756140C3942B
:10090D0004400375610075BB0822E5612410500297
:10091D0074FFF5617982B70402213EC3A861E52415
:10092D00985002A824C3E895634002A863882588DF
:10093D0026E570B4070375BB1022743279A787F0D2
:10094D00A4C5F0A2F733F8C3E895614002A8618809
:10095D00228824882588268864227540007541F0F8
:10096D0022C2AF75C820A8CCA9CDAA3A30CF010AB2
:10097D0075C824D2AFAB3BAC3C883B893CC3E89BEC
:10098D00F8E99C206908F9306602417F21D9AD3D17
:10099D008A3DF9EA9DFA600678FF79FF21BEAE3EE9
:1009AD00AF3F8B3E8C3FA83BA93CC3E89EF8E99F27
:1009BD00F9C3E54113FBE54013FAE82AF540E93B9D
:1009CD00F54150067540FF7541FF4126AA40AB41E8
:1009DD00AC40AD417E047F02C3EB9404400D1E1F5D
:1009ED00C3EB94084005206A021E1FC3ED13FDECF6
:1009FD0013FCDEF7C3EA9CFAEB9DFBEF6009C3E93C
:100A0D0013F9E813F8DFF7EA28FAEB39FB8A408B84
:100A1D004150067BFF8B408B41C3EB94025002D2B9
:100A2D00663069047F0341517892E6FFC3E5379440
:100A3D008240110FC3E53794A040010FC3EF940618
:100A4D0040027F057E02E541C4540FF9E541C454CF
:100A5D00F0F8E540C4540F28F8C3E89EFAE9940075
:100A6D00FB4009C3EA9402EB940050047A02E4FBC4
:100A7D0041CBAA40AB41EBC4FEEAC4540F4EFCC3BC
:100A8D00EA9CFAEB9400FBC3E813C313F8EA28FAC7
:100A9D00EB3400FB8A408B41C3EB94024002C266EB
:100AAD007802EBC4FE7B00EAC4540F4EFAC3EA98F9
:100ABD00FA4005C3940250027A027892E6FF306044
:100ACD000241CB855192855293D26043E680C3E4B7
:100ADD009AF8E49BF93066026157E8FAE9FBD3E92D
:100AED0013FDE813FC88518952C3EF94036038EF6E
:100AFD0020E00DE82CF8E93DF9ECFAEDFB020B20B6
:100B0D00E828F8E939F9C3E82402F8E93400F97A5C
:100B1D00FE7BFFC3EF9403400E8A538B54884D899F
:100B2D004E8C4F8D50618B885389548A4D8B4E8CD2
:100B3D004F8D503069127553F07554FF754FF07528
:100B4D0050FF7551F07552FF618BE8FAD3E813FC35
:100B5D008851C3EF94036020EF20E007E82CF8ECF8
:100B6D00FA6177E8282402F87AFEC3EF940340086F
:100B7D008A53884D8C4F618B88538A4D8C4FE56815
:100B8D00C3335002646BF5683060026195753402B1
:100B9D00D26043E680E52D54066034A840A941C3D8
:100BAD00E913F9E813F8C3E913F9E813F830690408
:100BBD00E92440F9C2AF53E67F759100C3E498F57F
:100BCD0094E499F595759104D26043E680D2AF22F5
:100BDD00D264754300752000306C03752040020B04
:100BED00FCD264754300752040306C03752000788D
:100BFD00017901206620E52D54066002C264791446
:100C0D00E541C313700104F8C39414400278143005
:100C1D006904781B791B206010E543600C30690373
:100C2D00D53404D26D81A6719D0543E59B5440B525
:100C3D002002819030690908C3E899400118812389
:100C4D0020640A08C3E899400261FC8123C264C292
:100C5D00AF53E67F7591003066127594007595F867
:0E0C6D00759104D26043E680D2AF61FCE54190
:100C7B007EFFC3334005C3334001FEC3E49E75942E
:100C8B0000F595816DC3E5339401500261FC30642E
:100C9B000261FCD80281A48123C26DC2AF53E67FEF
:100CAB00759100855394855495759104854D928566
:100CBB004E93D26043E680D2AFE52D5406600820F8
:100CCB006A020533020CE2306D0D206C0A206407BA
:100CDB001581158102159A2278003064027801E59E
:100CEB003775F007A4F9E5F028F5F0E9A2F013A2A7
:100CFB00F113A2F213F537C394785003753778C309
:100D0B00E53795384008D265D295D293D2973060AB
:100D1B0002A119854F92855093D26043E680222021
:100D2B007D16C2AF754202C296D294306202C29354
:100D3B00D2AF759F11020F1AC2AF754202C296D283
:100D4B0092306202C295D2AF759F11020F1A3072A8
:100D5B0043207D20C2AF75420390013A757B40D290
:100D6B0093C292306204C297A177D296D2AF759F8D
:100D7B0013020F1AC2AF75420390013A757B40D232
:100D8B0095C294306204C297A197D296D2AF759F49
:100D9B0010020F1A207D17C2AF754203900115D2B6
:100DAB0093306202C297D2AF759F13020F1AC2AF74
:100DBB00754203900115D295306202C297D2AF757E
:100DCB009F10020F1A207D16C2AF754204C294D237
:100DDB0092306202C297D2AF759F10020F1AC2AF48
:100DEB00754204C292D294306202C297D2AF759F01
:100DFB0013020F1A307243207D20C2AF754205904B
:100E0B000129757B10D297C296306204C295C11D21
:100E1B00D294D2AF759F11020F1AC2AF75420590D3
:100E2B00014B757B04D297C296306204C293C13DCD
:100E3B00D292D2AF759F11020F1A207D17C2AF75D8
:100E4B00420590010BD297306202C295D2AF759FCB
:100E5B0011020F1AC2AF75420590011FD297306273
:100E6B00EBC293D2AF759F11020F1A207D16C2AF42
:100E7B00754206C292D296306202C295D2AF759F6E
:100E8B0013020F1AC2AF754206C294D29630620299
:100E9B00C293D2AF759F10020F1A307244207D207F
:100EAB00C2AF75420190014B757B04D295C2943051
:100EBB006204C293C1C3D292D2AF759F10020F1AB4
:100ECB00C2AF754201900129757B10D293C292304B
:100EDB006205C295020EE4D294D2AF759F13020F36
:100EEB001A207D17C2AF75420190011FD295306257
:100EFB0002C293D2AF759F10020F1AC2AF75420197
:100F0B0090010BD293306202C295D2AF759F13C280
:100F1B006522900109757B00D295D293D297C2942A
:100F2B00C292C296C2622278807609087609087648
:100F3B00040876FF0876030876FF08760A0876031E
:100F4B00087601087601788C76010876FF0876FF23
:100F5B000876FF0876FF0876FF0876030876FF0809
:100F6B0076FF0876FF0876250876D008762808766F
:100F7B00500876040876FF08760208760008767A21
:100F8B000876FF08760108760108760008760308D4
:100F9B007600227887E6FFC272BF0302D27278888E
:100FAB00E6C394036008C27DE630E102D27DC27EC7
:100FBB007889E630E102D27EC3EF94026008758E29
:100FCB0001D273020FD6758E00C273227880E6149D
:100FDB009000809378A5F67881E614900080937842
:100FEB00A6F67886E61490008D9378A7F67886E6B9
:100FFB00F539C394025003753902789CE67538FFB6
:10100B00B402037538A0B4030375388278A3E614D1
:10101B0090009A93F566120F1D22227896E6FA78C5
:10102B0097E6FB7888E6B40305C3EB940EFB307FA1
:10103B00047A007BFFC3EB9AFCC3948250027C8240
:10104B007572000572EC8572F0A4C3E5F0947D40D7
:10105B00F222D27F11261205AB1205AB7A007B0070
:0F106B007C101205A1E55C2AFA74003BFBDCF354
:10107A007C04C3EB13FBEA13FADCF7FEC27F1126EA
:10108A0022757C00757D00E5EF20E60375200005DA
:10109A0020903FFFE520146006901DFF1460009326
:1010AA0004600375EF1653D9BF7581C043FF8012E0
:1010BA00059C75EF0643B203E5B3240220E70DF55C
:1010CA0021E5E320E0068521B343E301120F1D75F4
:1010DA0080FF75A40075F1B275D4DF7590A975A566
:1010EA00FC75F2FE75D50175A60175E241120F1D58
:1010FA00E4F8F6D8FD756801120F321215EB7898EC
:10110A008673753001C2AF1205B51205C51205AB5B
:10111A001205CC1205AB1205D31205ABC2AF757C12
:10112A0000757D0078FA79FA308507D9FBD8F7027D
:10113A001C00120F9E120FD711251126789886735C
:10114A00120F1D75881075890275C824759104756A
:10115A00D84075A82275B80275E690759B80759D72
:10116A000075D10E75BC5875BB0875BA1175E88043
:10117A0012059CD2AF1208A975360053DACF207E29
:10118A000343DA20307E0343DA1043DA01C2D8C2BD
:10119A00711205B5D2617B037A0CE55B70077A0C94
:1011AA00DB030211261205AB207003021126C2705E
:1011BA00E55CC3940240E1E52F541F855E5DF55E50
:1011CA00B55DD5DAD5C26153DACF207E0343DA2082
:1011DA00307E0343DA10C2D8C27178A2E67008D210
:1011EA0074E52F54E0F52FC2757529001205B03049
:1011FA007409C3E529940A4002D2751205A178023E
:10120A003074027800C3E55C9840F0C2AF1205C59D
:10121A001205C51205C5D2AF1205B5754C007888FE
:10122A00E6B40302611B1205A1788CE6C39401504F
:10123A000302131BE530C39401500302131B757C90
:10124A00A5757DF1207435C3E55C94FF5003021344
:10125A001BC2AF1205DAD2AF1205B0C3E55C940126
:10126A0050EFC2AF1205C51205A61205C5D2AF12BC
:10127A0005B0C3E55C94FF40E90217A37F02D27F61
:10128A0011261205B0C2AFC27F1126AE5CC3E55C5F
:10129A00947FD2AF5002612B12059CC2AF1205DABD
:1012AA00D2AFDFDA115DC3EE7897F61205B51217E1
:1012BA00267F0AD27F11261205B0C2AFC27F11263D
:1012CA00AE5CC3E55C947FD2AF50E612059CC2AF18
:1012DA001205C51205A61205C5D2AFDFD6115DEEFD
:1012EA0024037896F6F87997E7C3948240039850D6
:1012FA0006E824827897F61205B5121639121755A0
:10130A001205B01126C3E55C94FF5002414802174A
:10131A00A3757C00757D00C3E55C954C4003855C34
:10132A004C1205B078017988E7B403027805C3E561
:10133A005C9840024128C2AF1205DA1205DA12059A
:10134A00DAD2AF1205B5753000E4F531F532053160
:10135A00E531F4703F0532789AE67819146012780C
:10136A003214600D787D14600878FA1460037532BF
:10137A0000C3E53298401D120F1D12059C153275E7
:10138A00310078998673C2AF1205DAD2AF7898869F
:10139A00731205B01205A6E52A70053074022126DB
:1013AA0078012074027806C3E55C9840A17888E643
:1013BA00C3940360031205B0E52A7003021126C222
:1013CA00AF120F1DE4F522F523F524F525F526F5D0
:1013DA0067D2AF7885E6C333F565E4F544F545F59C
:1013EA0046F547F548F570F52CF52DF53775700873
:1013FA0075BB1012059C1208AD30EDFDA8BDA9BE43
:10140A00E97001F888711208B175700875BB10127D
:10141A000F9EC2AF7561FF1209478522618522625C
:10142A00852263D2AF7522017524017525017526BF
:10143A0001856069756A017888E6B40307C27D3060
:10144A007602D27DD268D269753300120E76120EF8
:10145A00A512096712096E12096712096E12096745
:0F146A00120BEE1206BB120CE3120D2A12096EC2
:10147900120BDD306E031207172066031208633062
:101489006603120893120CE3120D5912096E120B1E
:10149900EE306E0312074C120CE3120DD012096ED6
:1014A900120BDD306E031207AA120CE3120DFF12A4
:1014B900096E120BEE306E03120807120CE3120EBE
:1014C9007612096E1208AD120BDD120CE3120EA58D
:1014D9001208B112096E30693285646185646285CA
:1014E9006069756A0179187A0CC3E53399400FC2AE
:1014F90069D26A8A35856461856463021514C3E516
:101509005C9401400302146A0215A2306A25206C1A
:1015190022E535147006C26AD26B816AF535C3E5D6
:101529005C9401400302146A7888E6C3940360035B
:101539000215A275360078FA79A4E760027803C328
:10154900E55F985054307404E52A604D7888E6B414
:101559000317207D05207607A172307602A172203B
:101569006C07D26C85646181A978F0306C0585645B
:10157900617820C3E541985002816A306C1BC26CC6
:10158900C27D307602D27DD26A7535128564618159
:101599006A0536E55C6002A1A5753600C2AF120F77
:1015A9001D7887E6FE7602120F9E7887EEF6E4F53F
:1015B90022F523F524F525F526F565752C00752DFD
:1015C90000D2AF1205B0120F1D78A4E66006C295CD
:1015D900C297C293307409C3E536940440022126A8
:1015E9006153901A0D782012167BE520B4550CA38F
:1015F90012167BE520B4AA03021619757CA5757D20
:10160900F1120F32121639757C00757D00021638F9
:10161900901A0378807B0A12167BA308DBF9901ACB
:101629000F788C7B1912167BA308DBF9901A2822F4
:10163900C2AF1216BE12169B901A00740E121680B3
:10164900A37409121680A37415121680901A0378D0
:10165900807B0A12167FA308DBF9901A0F788C7B1E
:101669001912167FA308DBF91216D11216AF901AB8
:101679002822E493F622E6438F01538FFDFFC3E549
:1016890083941C400122EF857CB7857DB7F0538F89
:10169900FE22438F02438F01857CB7857DB7901A5F
:1016A9000DF0538FFC22901A0D7455D180901A0EAB
:1016B90074AAD180227A3079D07820901A40D17BCF
:1016C900E520F709A3DAF7227A3079D0901A40E7B2
:1016D900D18009A3DAF922AB74A875BB010279801C
:1016E900BB02027981BB03027982BB04027984BB04
:1016F90005027986BB06027992BB07027987BB0886
:101709000279A3BB0902799CBB0A027988BB0B0247
:101719007989E8F7227C051205B5DCFB22C2AF12F4
:1017290005C51205CC1205D31205DA1205A6120554
:10173900C51205CC1205D31205DA1205A61205C584
:101749001205CC1205D31205DAD2AF22C2AF1205A7
:10175900DA1205D31205CC1205C51205A61205DA4F
:101769001205D31205CC1205C51205A61205DA1207
:1017790005D31205CC1205C5D2AF22AE74AF75C21E
:10178900AF1205C51205C51205C51205A6DEF2126E
:1017990005DA1205A6DFF8D2AF22F126F11EF11EF5
:1017A900757401757501757600F1847C05AD5C125F
:1017B90005B5C3ED955C70F5C3E55C9401400AC3BA
:1017C900E55C94FF40320217DFD1E0D139F126C23E
:1017D900AF75EF16F11EDCD50576C3E57694035097
:1017E9000280C6F11E0575E5741490009F93F808F0
:1017F900C3E57598500280AE12171E12171E0574A4
:10180900C3E574940C5002809A120F32121639C231
:07181900AF75EF1612171E58
:0319FD0002108B4A
:101A00000E0915090904FF03FF0A03010155AA0184
:101A1000FFFFFFFFFF03FFFFFF25D0285004FF0259
:091A2000007AFF0101000300FF40
:101A400023526F746F724765656B73323041232088
:101A500023424C48454C4923463333302320202031
:101A60002020202020202020202020202020202076
:101C0000C2AFC2D353D9BF7581C043B20343FF8073
:101C1000752438752503B1DC7529A5752AF175E29F
:101C20004043F12053A4DF75D4FFD2857DFA7803B9
:101C300079E67C10752200752300901DE97B0675FE
:101C400024987525013085028145208508D8FBD967
:101C5000F9DCF781B7308508D8FBD9F9DCF781B713
:101C6000B19CE493A3C39A6004DDC381B7DBDBB10D
:101C70008E6002812E7B08E493FAA3B16FDBF87AC1
:101C800030B16F752200752300B18EEAFCEBFDC305
:101C9000ED94FE400EB18E8A278B28ED30E0048A49
:101CA000828B83B18E7AC270D8C3ED94FE601950D6
:101CB000CEBD002BEC600F7520007521FF7529004B
:101CC000752A000200008100A827A9280809D80465
:101CD000D90281DCB192EA89AAF281CE0D81A3C337
:101CE000ED94035053EDA2E092007AC5C3E58294CF
:101CF00000E583941C508A200010438F02438F011B
:101D00008529B7852AB7F0300029A827A92808090E
:101D1000438F01538FFDD804D902A133C3E58394C7
:101D20001C4003A3A11689AAE28529B7852AB7F02A
:101D3000A3A116538FFC817F7AC1BD030CE493A34A
:101D4000FAB153DCF8B14B817F8181AA22AB23B178
:101D50006FEBFAEA6222752608C3E52313F523E543
:101D60002213F52250066323A0632201D526EAB18F
:101D7000DCB1DC75260AEAF4200102D285300102CA
:101D8000C285B1DCC3134002C201D526EB22B19259
:101D9000EAFB208502A192308502A197752608AE44
:101DA00024AF25C3EF13FFEE13FEB1E0B1DCC3EAAD
:101DB000133085024480FA30E703632201C3E52330
:101DC00013F523E52213F52250066323A0632201B5
:101DD000D526D9E52265236523F52222AE24AF2539
:101DE0000E0FDEFEDFFCD20122424C48656C6934E6
:071DF000373164F3300601F6
:00000001FF
